:020000020000FC
:100000001EC00AE02095089410F4C49A02C0C49857
:10001000000005D004D026950A95B1F7089511E1A6
:100020001A95F1F708951FEF1A95F1F708956FEFFC
:1000300070E27A95F1F770E26A95D9F708951FE9B1
:100040001DBFC49ABC9AC19AB99A3E983D98379AF6
:1000500035983298319830983998389AC198E7DFB6
:10006000C19A38E23A95F1F7369A3699FECF44B103
:1000700055B1C198242FC5DF252FC3DF21E0C1DF93
:0E00800022E0BFDF23E0BDDF24E0BBDFE7CFDF
:00000001FF
